:030000000219FDE5
:03000B000200AA46
:03002B0002015C73
:03005B000202F0AE
:030073000202DDA9
:1000800002030406080C10182030406080040608A3
:100090000C10182030406080A0C00003070F1F0D17
:1000A0000D04050D050305030302C2AFC0D0C0E077
:1000B000206214E5256009E473E525F4F58AD2622F
:1000C000D0E0D0D0D2AF3285268AC262E526F46075
:1000D0002F30682520720DD0E0D0D0D297D295D2A3
:1000E00093D2AF32D297D295D293206F0C2065096C
:1000F000740AD5E0FDE57B4290D0E0D0D0D2AF329B
:10010000758A00C28DD26201F901B9306805206597
:1001100002C29701B9306805206502C29501B93065
:100120006805206502C29301B9C29630680A20654D
:10013000077408D5E0FDC29701B9C29430680A205F
:1001400065077408D5E0FDC29501B9C29230680A0E
:100150002065077408D5E0FDC29301B9C2AFC2ADF6
:1001600053E6EFC0D0C0E0D2D3D2AFC2CEE52A6012
:1001700007207449152A21BD7800790020742EE5E6
:1001800080307E01F430E50278FF53DACF207E0321
:1001900043DA20307E0343DA10C2D8C271E58030E2
:1001A0007E01F430E50279FFC3E89970CB3061033A
:1001B000752A18207403752A18885CD27020740D73
:1001C000E52B6004152B21CD43DA01C2D820700243
:1001D000413CA85C206102C2702074367982B70469
:1001E00031C3E894F0400374F0F8E8C4540F28F8E1
:1001F0007984B703024112C313C313872120080275
:10020000C313200A06C3C898F8411228F850037493
:10021000FFF88822E52D54066022206B1FE536C3C7
:1002200033C333F8E564C313C313F9C39522400203
:100230008922E82522F52250037522FF7882B60430
:1002400059852224A824C3E52495614002A861C3EE
:10025000E895634002A8638825E5667002418DC376
:10026000E8AA669A5003E8FAE4F9EAC333FBE568C2
:10027000F45B29400D2567F8E56760021567400BC0
:10028000418D0AC3E5679A5002056778FF8826C248
:100290006FC3E52694F84002D26F20CF0AD0E0D099
:1002A000D043E610D2AD32C2CF053A7801E52A60DC
:1002B00005307402152AC3E55C94014005755F00A2
:1002C00041D3756000756900E55F2401F55F500357
:1002D000755FFFD0E0D0D043E610D2AD32C2AF534D
:1002E000E67F7592FA7593FFC260759104D2AF32C2
:1002F000C2AF53E6EFC2ADC0D0C0E0C0F0D2D3D29F
:10030000AFA8FBA9FCC2D8307102615753DACF20E5
:100310007E0343DA10307E0343DA20D271E5803069
:100320007E01F420E502612E88278928A18453DA12
:10033000CF207E0343DA20307E0343DA10C2D8C2D6
:1003400071307402A1707800E580307E01F430E5F0
:1003500002A170885CA15853DACF207E0343DA20D3
:10036000307E0343DA10C271206102813053DACF4C
:10037000207E0343DA10307E0343DA20C2D8D271E4
:1003800088578958C3E89555F8E99556F97B007E5A
:10039000087A00C3E8948CE994005005755B0081ED
:1003A00022882178A2E6A8216055C3E894C8E99480
:1003B000005008E4D2E4FB7A0A61FDC3E89468E9DE
:1003C00094015008E4D2E3FB7A0F61FDC3E894D0B6
:1003D000E994025008E4D2E2FB7A1E61FDC3E8947E
:1003E000A0E994055008E4D2E1FB7A3C61FDC3E842
:1003F0009498E994085008E4D2E0FB7A787E00C330
:10040000E89559FCE9955AFD30E70AECF42401FC23
:10041000EDF43400FD755B00C3EC9AED9E5003755E
:100420005B018859895A8557558558567802A158D5
:10043000C3E89527F8E99528F9307C02A13C307B88
:1004400002A13C307A02A1352075028153E9FDE812
:10045000FC8172E9C313F9E813F8307902A135E998
:10046000C313F9E813F8307802A135E9C313FDE8A6
:0E04700013FC20612CC3EC941CED940240029E
:10047E008189ED701EC3EC94C850180529E52970CA
:10048E00021529C3E529940A5002A170755C00D2A9
:10049E0070A170E529600215297888E6F9740020AC
:1004AE007F087896B90302789EE624FAFEE43400BB
:1004BE00FFC3EC9EFCED9FFD9208B90310A20850FD
:1004CE0007207609D27681DB307602C276A20850FA
:1004DE0016B9030DECF42401FCEDF43400FD020416
:1004EE00F578007900A13CB90315EC33FCED33FD32
:1004FE00C3EC940AFCED9400FD50047C007D00C317
:10050E00EC94FFED9400400678FF7900A13CEC8559
:10051E0072F0A4C5F0A2F733F87900400302055833
:10052E0078FF7900020558E9C313F9E813F8307C17
:10053E000EE9600278FFC3E81338F8E43400F9C31B
:10054E00E894FFE99400400278FF885CD270206145
:10055E0002A170741FF4552F4BF52FC274EB70026D
:10056E00D274752A18307403752A0A306102A18478
:10057E0020740353DAFE207403752B06D0F0D0E0FE
:10058E00D0D0D2AD43E6103279010205B479030220
:10059E0005B4790A0205B4791E0205B47964020520
:1005AE00B479C80205B47817E4D5E0FDD8FAD9F6C7
:1005BE00227A147B780205DB7A107B8C0205DB7ABB
:1005CE000D7BB40205DB7A0B7BC80205DBE573D528
:1005DE00E001227902E4C294D5E0FDC295D5E0FD9A
:1005EE00D295D5E0FDD294D5E0FDE920E002C29788
:1005FE0030E002C293E573D5E0FDE920E002D29728
:10060E0030E002D2937496D5E0FDD9C9EAF8D5E070
:10061E00FDD8FBDBB8C29422C37C007D0075F000D0
:10062E0005F0EA33FAEB33FB50F6EB13FBEA13FA61
:10063E00C3E9FFE8FEE89AF8E99BF95004EFF9EEFA
:10064E00F8B3EC33FCED33FDD5F0DFEDF9ECF82229
:10065E00E889F08A20D2D4F8A9F07B0030F70B7B22
:10066E00FFF42401F8E9F43400F9E88520F0A4AD94
:10067E00F0F8E98520F0A4AFF0FEED2EF974003FFE
:10068E00FA7C04C3EA13FAE913F9E813F8DCF48BE5
:10069E00F030F70AE8F42401F8E9F43400F9E889B7
:1006AE00F0C2D4F8A9F0227882B60403020710C370
:1006BE00E55C940140030206DA852224E4F544F554
:1006CE0045F546F547F548C26E0207107882E6FCFE
:1006DE00D26EE522F523783879C7AA40AB41C3EB39
:1006EE0013FBEA13FAEC146013C3EB13FBEA13FAD1
:1006FE00EC14146007C3EB13FBEA13FAD1268844FB
:10070E00894522C3E5449523F8E5459400F9500C3C
:10071E00C3E89480E994FF4016020741C3E8947F32
:10072E00E994005003020741787F7900020741786F
:10073E008079FF8849894A22E5492546F8E54A35F8
:10074E0047F9854A20E4300701F43548FA30E709C5
:10075E00C3EA94F0401502077FC3EA940F500302D8
:10076E00077F78FF79FF7A0F02077F780079007A8A
:10077E00F0C3E5249561500AC374019524500B0211
:10078E00079DE54A20E70E02079DE54A30E70688F9
:10079E004689478A482278A5E6FAC3E54933F8E543
:1007AE004A33F9D15EE930E70BC3E89480E994FF50
:1007BE004013E1D7C3E8947FE994005002E1D77863
:1007CE007F7900E1D7788079FFE820E715C3E5232C
:1007DE0098F84009C3E8940140030207FE7801022D
:1007EE0007FEE8F424012523F840030207FE78FFF4
:1007FE00884B2278A6E6FAA847A94812065EE93089
:10080E00E70CC3E89401E994FF4016020833C3E8ED
:10081E0094FFE99400500302083378FF7900020830
:10082E0033780179FFE920E715C3E54B98F84009C5
:10083E00C3E89401400302085A780102085AE8F40A
:10084E002401254BF8400302085A78FF88242278A9
:10085E00FF20692879A1E76023E541601F74FF85B9
:0E086E0041F0848539F0306A0375F005A4F876
:10087C00C5F0600278FFC3E895645002A8648863F1
:10088C0022C3E5409440E5419401E5635003140113
:10089C009E046002F563220208A62275E890227875
:1008AC0083E6FF30EDF9A8BDA9BE0570C3E57094D1
:1008BC00084052757000E9FA79A0E76044EA7007C5
:1008CC00E571601B0208DFC3E895716010E571509B
:1008DC0006600C140208EB0460F90208EBE571F5F4
:1008EC0071C3946D401B7561C0C394044013756152
:1008FC0080C39404400B756140C39404400375613C
:10090C000075BB0822E5612410500274FFF5617973
:10091C0082B704022138C3A861E524985002A824A8
:10092C00C3E895634002A86388258826E570B40760
:10093C000375BB1022743279A787F0A4C5F0A2F717
:10094C0033F8C3E895614002A86188228824882581
:10095C0088268864227540007541F022C2AF75C8A4
:10096C0020A8CCA9CDAA3A30CF010A75C824D2AFA1
:10097C00AB3BAC3C883B893CC3E89BF8E99C2069C9
:10098C0008F9306602417721D1AD3D8A3DF9EA9DE7
:10099C00FA600478FF79FFAE3EAF3F8B3E8C3FA8E8
:1009AC003BA93CC3E89EF8E99FF9C3E54113FBE57D
:1009BC004013FAE82AF540E93BF54150067540FF33
:1009CC007541FF411EAA40AB41AC40AD417E047F56
:1009DC0002C3EB9404400D1E1FC3EB94084005208A
:1009EC006A021E1FC3ED13FDEC13FCDEF7C3EA9C79
:1009FC00FAEB9DFBEF6009C3E913F9E813F8DFF795
:100A0C00EA28FAEB39FB8A408B4150067BFF8B407E
:100A1C008B41C3EB94025002D2663069047F0341D0
:100A2C00497892E6FFC3E537948240110FC3E5374E
:100A3C0094A040010FC3EF940640027F057E02E5AF
:100A4C0041C4540FF9E541C454F0F8E540C4540FC7
:100A5C0028F8C3E89EFAE99400FB4009C3EA940223
:100A6C00EB940050047A02E4FB41C3AA40AB41EB87
:100A7C00C4FEEAC4540F4EFCC3EA9CFAEB9400FB90
:100A8C00C3E813C313F8EA28FAEB3400FB8A408B53
:100A9C0041C3EB94024002C2667802EBC4FE7B00B9
:100AAC00EAC4540F4EFAC3EA98FA4005C3940250B4
:100ABC00027A027892E6FF30600241C3855192853A
:100ACC005293D26043E680C3E49AF8E49BF9306613
:100ADC0002614FE8FAE9FBD3E913FDE813FC8851F6
:100AEC008952C3EF94036038EF20E00DE82CF8E94D
:100AFC003DF9ECFAEDFB020B18E828F8E939F9C3DB
:100B0C00E82402F8E93400F97AFE7BFFC3EF940382
:100B1C00400E8A538B54884D894E8C4F8D50618377
:100B2C00885389548A4D8B4E8C4F8D503069127579
:100B3C0053F07554FF754FF07550FF7551F07552A9
:100B4C00FF6183E8FAD3E813FC8851C3EF94036088
:100B5C0020EF20E007E82CF8ECFA616FE82824027B
:100B6C00F87AFEC3EF940340088A53884D8C4F618A
:100B7C008388538A4D8C4FE568C3335002646BF500
:100B8C0068306002618D753402D26043E680E52DD9
:100B9C0054066034A840A941C3E913F9E813F8C31B
:100BAC00E913F9E813F8306904E92440F9C2AF53AA
:100BBC00E67F759100C3E498F594E499F5957591E9
:100BCC0004D26043E680D2AF22D264754300752014
:100BDC0000306C03752040020BF4D2647543007531
:100BEC002040306C0375200078017901206620E5E7
:100BFC002D54066002C2647914E541C313700104DC
:100C0C00F8C3941440027814306904781B791B20C3
:100C1C006010E543600C306903D53404D26D819EBD
:100C2C0071950543E59B5440B520028188306909D4
:100C3C0008C3E899400118811B20640A08C3E8998D
:100C4C00400261F4811BC264C2AF53E67F75910010
:100C5C003066127594007595F8759104D26043E670
:0F0C6C0080D2AF61F4E5417EFFC3334005C3334F
:100C7B004001FEC3E49E759400F5958165C3E53391
:100C8B009401500261F430640261F4D802819C81BA
:100C9B001BC26DC2AF53E67F75910085539485548B
:100CAB0095759104854D92854E93D26043E680D223
:100CBB00AFE52D54066008206A020533020CDA30CA
:100CCB006D0D206C0A206407158115810215892290
:100CDB0078003064027801E53775F007A4F9E5F088
:100CEB0028F5F0E9A2F013A2F113A2F213F537C322
:100CFB0094785003753778C3E53795384008D2653B
:100D0B00D297D295D293306002A111854F92855024
:100D1B0093D26043E68022207D16C2AF754202C299
:100D2B0094D296306202C293D2AF759F10020F110C
:100D3B00C2AF754202C294D292306202C297D2AF56
:100D4B00759F10020F11307243207D20C2AF754288
:100D5B000390013A757B10D293C292306204C29514
:100D6B00A16FD294D2AF759F13020F11C2AF754210
:100D7B000390013A757B10D297C296306204C295EC
:100D8B00A18FD294D2AF759F11020F11207D17C284
:100D9B00AF754203900115D293306202C295D2AF68
:100DAB00759F13020F11C2AF754203900115D297B5
:100DBB00306202C295D2AF759F11020F11207D16C2
:100DCB00C2AF754204C296D292306202C295D2AFC4
:100DDB00759F11020F11C2AF754204C292D29630A9
:100DEB006202C295D2AF759F13020F11307243206E
:100DFB007D20C2AF754205900129757B40D295C20B
:100E0B0094306204C297C115D296D2AF759F10026F
:100E1B000F11C2AF75420590014B757B04D295C281
:100E2B0094306204C293C135D292D2AF759F100237
:100E3B000F11207D17C2AF75420590010BD2953073
:100E4B006202C297D2AF759F10020F11C2AF7542EB
:100E5B000590011FD2953062EBC293D2AF759F10F4
:100E6B00020F11207D16C2AF754206C292D294308A
:100E7B006202C297D2AF759F13020F11C2AF7542B8
:100E8B0006C296D294306202C293D2AF759F110202
:100E9B000F11307243207D20C2AF75420190014B80
:100EAB00757B04D297C296306204C293C1BBD292B7
:100EBB00D2AF759F11020F11C2AF7542019001297C
:100ECB00757B40D293C292306204C297C1DBD2963B
:100EDB00D2AF759F13020F11207D17C2AF75420160
:100EEB0090011FD297306202C293D2AF759F11024D
:100EFB000F11C2AF75420190010BD293306202C247
:100F0B0097D2AF759F13C26522900109757B00D2F2
:100F1B0097D295D293C296C294C292C26222788023
:100F2B0076090876090876040876FF0876030876B2
:100F3B00FF08760A087603087601087601788C7626
:100F4B00010876FF0876FF0876FF0876FF0876FF24
:100F5B000876030876FF0876FF0876FF08762508E3
:100F6B0076D00876280876500876040876FF08763F
:100F7B000208760008767A0876FF08760108760173
:100F8B00087600087603087600227887E6FFC2729F
:100F9B00BF0302D2727888E6C394036008C27DE671
:100FAB0030E102D27DC27E7889E630E102D27EC387
:100FBB00EF94026008758E01D273020FCD758E000F
:100FCB00C273227880E6149000809378A5F678811E
:100FDB00E6149000809378A6F67886E61490008D40
:100FEB009378A7F67886E6F539C3940250037539E2
:100FFB0002789CE67538FFB402037538A0B403037E
:10100B0075388278A3E61490009A93F566120F1444
:10101B0022227896E6FA7897E6FB7888E6B4030501
:10102B00C3EB940EFB307F047A007BFFC3EB9AFC7F
:10103B00C3948250027C827572000572EC8572F04B
:10104B00A4C3E5F0947D40F222D27F111D1205A5B9
:10105B001205A57A007B007C1012059BE55C2AFA31
:0F106B0074003BFBDCF37C04C3EB13FBEA13FACA
:10107A00DCF7FEC27F111D22757C00757D00E5EF4D
:10108A0020E6037520000520903FFFE52014600646
:10109A00901DFF1460009304600375EF1653D9BFC7
:1010AA007581C043FF8012059675EF0643B203E5CA
:1010BA00B3240220E70DF521E5E320E0068521B3FC
:1010CA0043E301120F147580FF75A40075F1B27520
:1010DA00D4DF7590A975A5FC75F2FC75D50175A6C6
:1010EA000175E241120F14E4F8F6D8FD7568011291
:1010FA000F291215DA78988673753001C2AF120576
:10110A00AF1205BF1205A51205C61205A51205CD17
:10111A001205A5C2AF757C00757D0078FA79FA30A0
:10112A008507D9FBD8F7021C00120F95120FCE11B2
:10113A001C111D78988673120F1475881075890210
:10114A0075C82475910475D84075A82275B80275BA
:10115A00E690759B80759D0075D10E75BC5875BB60
:10116A000875BA1175E880120596D2AF1208A375F0
:10117A00360053DACF207E0343DA20307E0343DA87
:10118A001043DA01C2D8C2711205AFD2617B037A69
:10119A000CE55B70077A0CDB0302111D1205A52012
:1011AA00700302111DC270E55CC3940240E1E52F91
:1011BA00541F855E5DF55EB55DD5DAD5C26153DA39
:1011CA00CF207E0343DA20307E0343DA10C2D8C22E
:1011DA007178A2E67008D274E52F54E0F52FC27533
:1011EA007529001205AA307409C3E529940A400238
:1011FA00D27512059B78023074027800C3E55C98B8
:10120A0040F0C2AF1205BF1205BF1205BFD2AF121E
:10121A0005AF754C007888E6B40302611212059B8B
:10122A00788CE6C394015003021312E530C394018B
:10123A005003021312757CA5757DF1207435C3E540
:10124A005C94FF5003021312C2AF1205D4D2AF123C
:10125A0005AAC3E55C940150EFC2AF1205BF12059F
:10126A00A01205BFD2AF1205AAC3E55C94FF40E9FC
:10127A000217867F02D27F111D1205AAC2AFC27F52
:10128A00111DAE5CC3E55C947FD2AF50026122129D
:10129A000596C2AF1205D4D2AFDFDA1154C3EE7885
:1012AA0097F61205AF1217097F0AD27F111D120590
:1012BA00AAC2AFC27F111DAE5CC3E55C947FD2AFF8
:1012CA0050E6120596C2AF1205BF1205A01205BF5D
:1012DA00D2AFDFD61154EE24037896F6F87997E761
:1012EA00C394824003985006E824827897F6120540
:1012FA00AF12161C1217381205AA111DC3E55C9409
:10130A00FF5002413F021786757C00757D00C3E5D8
:10131A005C954C4003855C4C1205AA78017988E7F4
:10132A00B403027805C3E55C984002411FC2AF12BC
:10133A0005D41205D41205D4D2AF1205AF75300008
:10134A00E4F531F5320531E531F4703F0532789A2A
:10135A00E67819146012783214600D787D146008EA
:10136A0078FA146003753200C3E53298401D120FF3
:10137A0014120596153275310078998673C2AF1228
:10138A0005D4D2AF789886731205AA1205A0E52A69
:10139A007005307402211D78012074027806C3E5B5
:1013AA005C9840A17888E6C3940360031205AAE515
:1013BA002A700302111DC2AF120F14E4F522F5239D
:1013CA00F524F525F526F567D2AF7885E6C333F51A
:1013DA0065E4F544F545F546F547F548F570F52C0D
:1013EA00F52DF53775700875BB101205961208A70A
:1013FA0030EDFDA8BDA9BEE97001F888711208ABED
:10140A0075700875BB10120F95C2AF7561FF12098E
:10141A0041852261852262852263D2AF75220175D8
:10142A002401752501752601856069756A01788828
:10143A00E6B40307C27D307602D27DD268D26975DE
:10144A003300120E6E120E9D1209611209681209FA
:10145A0061120968120961120BE61206B5120CDB59
:0F146A00120D22120968120BD5306E03120711F2
:1014790020660312085D30660312088D120CDB1218
:101489000D51120968120BE6306E03120746120C51
:10149900DB120DC8120968120BD5306E031207A4AE
:1014A900120CDB120DF7120968120BE6306E0312EB
:1014B9000801120CDB120E6E1209681208A7120B32
:1014C900D5120CDB120E9D1208AB12096830693275
:1014D900856461856462856069756A0179187A0C29
:1014E900C3E53399400FC269D26A8A35856461853B
:1014F900646302150BC3E55C9401400302146102A5
:101509001591306A1D206C1AE535147006C26AD22D
:101519006B8161F535C3E55C9401400302146102F6
:10152900159175360078FA79A4E760027803C3E566
:101539005F985054307404E52A604D7888E6B40306
:1015490017207D05207607A161307602A161206C04
:1015590007D26C85646181A078F0306C058564617F
:101569007820C3E5419850028161306C1BC26CC27E
:101579007D307602D27DD26A7535128564618161CA
:101589000536E55C6002A194753600C2AF120F14EE
:101599007887E6FE7602120F957887EEF6E4F52253
:1015A900F523F524F525F526F565752C00752D002F
:1015B900D2AF1205AA120F1478A4E66006C297C228
:1015C90095C293307409C3E53694044002211D6124
:1015D9004A901A0D782012165EE520B4550CA31214
:1015E900165EE520B4AA030215FC120F2912161C77
:1015F90002161B901A0378807B0A12165EA308DB79
:10160900F9901A0F788C7B1912165EA308DBF990F2
:101619001A2822C2AF1216A112167E901A00740E51
:10162900121663A37407121663A374151216639036
:101639001A0378807B0A121662A308DBF9901A0F45
:10164900788C7B19121662A308DBF91216B41216EC
:1016590092901A2822E493F622E6438F01538FFDD4
:10166900FFC3E583941C400122EF857CB7857DB7D4
:10167900F0538FFE22438F02438F01857CB7857D0E
:10168900B7901A0DF0538FFC22901A0D7455D1633F
:10169900901A0E74AAD163227A3079D07820901AE0
:1016A90040D15EE520F709A3DAF7227A3079D090A4
:1016B9001A40E7D16309A3DAF922AB74A875BB0113
:1016C900027980BB02027981BB03027982BB0402E1
:1016D9007984BB05027986BB06027992BB07027938
:1016E90087BB080279A3BB0902799CBB0A027988E6
:1016F900BB0B027989E8F7227C051205AFDCFB22D6
:10170900C2AF1205BF1205C61205CD1205D41205C6
:10171900A01205BF1205C61205CD1205D41205A0E7
:101729001205BF1205C61205CD1205D4D2AF22C2C9
:10173900AF1205D41205CD1205C61205BF1205A0B8
:101749001205D41205CD1205C61205BF1205A01245
:1017590005D41205CD1205C61205BFD2AF22AE744B
:10176900AF75C2AF1205BF1205BF1205BF1205A0A2
:10177900DEF21205D41205A0DFF8D2AF22F109F189
:1017890001F101757401757501757600F1677C05C4
:10179900AD5C1205AFC3ED955C70F5C3E55C9401D2
:1017A900400AC3E55C94FF40320217C2D1C3D11C81
:1017B900F109C2AF75EF16F101DCD50576C3E576FF
:1017C9009403500280C6F1010575E5741490009FD9
:1017D90093F808C3E57598500280AEF101F101054F
:1017E90074C3E574940C5002809C120F29D11CC259
:0617F900AF75EF16F101CF
:0319FD0002108253
:101A00000E0715090904FF03FF0A03010155AA0186
:101A1000FFFFFFFFFF03FFFFFF25D0285004FF0259
:091A2000007AFF0101000300FF40
:101A400023536B7977616C6B6572323041232020B0
:101A500023424C48454C4923463333302320202031
:101A60002020202020202020202020202020202076
:101C0000C2AFC2D353D9BF7581C043B20343FF8073
:101C1000752438752503B1DC7529A5752AF175E29F
:101C20004043F12053A4DF75D4FFD2857DFA7803B9
:101C300079E67C10752200752300901DE97B0675FE
:101C400024987525013085028145208508D8FBD967
:101C5000F9DCF781B7308508D8FBD9F9DCF781B713
:101C6000B19CE493A3C39A6004DDC381B7DBDBB10D
:101C70008E6002812E7B08E493FAA3B16FDBF87AC1
:101C800030B16F752200752300B18EEAFCEBFDC305
:101C9000ED94FE400EB18E8A278B28ED30E0048A49
:101CA000828B83B18E7AC270D8C3ED94FE601950D6
:101CB000CEBD002BEC600F7520007521FF7529004B
:101CC000752A000200008100A827A9280809D80465
:101CD000D90281DCB192EA89AAF281CE0D81A3C337
:101CE000ED94035053EDA2E092007AC5C3E58294CF
:101CF00000E583941C508A200010438F02438F011B
:101D00008529B7852AB7F0300029A827A92808090E
:101D1000438F01538FFDD804D902A133C3E58394C7
:101D20001C4003A3A11689AAE28529B7852AB7F02A
:101D3000A3A116538FFC817F7AC1BD030CE493A34A
:101D4000FAB153DCF8B14B817F8181AA22AB23B178
:101D50006FEBFAEA6222752608C3E52313F523E543
:101D60002213F52250066323A0632201D526EAB18F
:101D7000DCB1DC75260AEAF4200102D285300102CA
:101D8000C285B1DCC3134002C201D526EB22B19259
:101D9000EAFB208502A192308502A197752608AE44
:101DA00024AF25C3EF13FFEE13FEB1E0B1DCC3EAAD
:101DB000133085024480FA30E703632201C3E52330
:101DC00013F523E52213F52250066323A0632201B5
:101DD000D526D9E52265236523F52222AE24AF2539
:101DE0000E0FDEFEDFFCD20122424C48656C6934E6
:071DF000373163F3300601F7
:00000001FF
